:020000042000DA
:10000000C0440020E13D0020A13B0020A33B002094
:1000100000000000000000000000000000000000E0
:10002000000000000000000000000000A53B0020D0
:100030000000000000000000A73B0020A93B0020BA
:10004000513C0020533C0020553C0020613C0020E6
:10005000000000000000000000000000693C0020DB
:10006000753C0020773C0020C73C0020C93C0020A4
:10007000CB3C0020CD3C0020000000000000000030
:100080000000000000000000000000000000000070
:100090000000000000000000000000000000000060
:1000A0000000000000000000000000000000000050
:1000B0000000000000000000CF3C00200000000015
:1000C00038384D53313030000101000080B5CC226A
:1000D00092000021BD4801F083FC01BD80B5812262
:1000E00092000021BA4801F07BFC10220021B9489F
:1000F00001F076FC01BD80B550220021B64801F028
:100100006FFC01BDF1B586B0B4480068000A00027A
:1001100080B2B3490978084180B20490B1480469BB
:1001200000258020C00006990818039068462946DB
:10013000016001810E46012705E028003D00B54021
:1001400005436408761C202E2DDA3C42F5D0B00021
:1001500003990818019040880499884217DB684683
:100160004088401C6946488028003D00B540054352
:10017000300000F054F80100C90F0818401000F0DA
:1001800058F8202803D229003D0085400D430198EE
:100190004088694609888142D3D26946088068460A
:1001A00031000181CDE78E48694649880171694671
:1001B0000988C18068460089400106990818894964
:1001C000096889B20022134614460BE00E00F607B8
:1001D00006D56600865BB24202D2320023009BB293
:1001E0004910641C102CF1DB7D4843718560B748D1
:1001F00000210A460BE0EB0707D49300039CE318A9
:100200005B88834201D2180011006D08521C202A1D
:10021000F1DB734A51701146488007B0F0BD4128A8
:1002200002D30020C04370471A304D2800DB40380D
:10023000704701000D39402902D30020C0437047A8
:100240001A3800D540307047F3B589B0A048C06A6D
:10025000800B80B2002805D05C48017801220A4357
:100260000270B1E001F0F8FD002819D1002411E07E
:100270002100280001F0A0FB4000099909180A9A02
:10028000105A0A88801A08806D1C01F04CFB8542C8
:10029000EEDB641C01F04AFB844201DA0025F4E73E
:1002A0000020049003908B4800680100090A0A00AE
:1002B000D207D20F0792000B0007000F0690002014
:1002C0000290009050E00099019801F075FB400009
:1002D00009990E5E7E480021405EB04202DA059820
:1002E000401C0590300001F0FFFD0221784A515E6C
:1002F000814200DA7F1C0798002809D0102011469F
:10030000085EB04200DA641C7142884200DA6D1C5B
:100310000198401C019001F011FB01998142D2DB50
:100320000598002806D004980121009A91400143C5
:1003300089B20491002F06D003980121009A9140C0
:10034000014389B20391EDB20698854209DBE4B21C
:10035000844206DB02980121009A9140014389B250
:1003600002910098401C009001F0E0FA009981424F
:1003700006DA002005900746044605460190CAE7C4
:100380001248049981800399C180029901810299E0
:1003900089B2002904D0017802220A43027013E0D6
:1003A000049989B2002903D0017804220A4302701B
:1003B000039989B2002903D0017808220A43027008
:1003C0000A99099800F03BF80BB0F0BD3471002099
:1003D0006474002068760020787600206870002021
:1003E000D870002008000051F1B582B07F48416804
:1003F000890089080091006884B20025012700E087
:100400006D1C1E2D1ADA0098E8403840F8D00026FE
:1004100000E0761C102EF3DA2000F0403840F8D0CF
:100420002801801940000299085E01F05DFD7049C5
:100430000022895E8842ECDBB9480770F7BDF8B549
:10044000040001F076FA00281CD000273D0013E0DC
:10045000280001F0BBFA4000205EB2490022895E0C
:10046000814208DA012601F064FA401E2900401A90
:1004700086403E4337006D1C01F05BFA8542E7DBA6
:10048000A9480770F1BDF8B50700A8480688002400
:1004900011E022002900380000F01EF8002804D0E6
:1004A00022002900380000F043F96D1C01F046FAE3
:1004B0008542EEDB641C01F039FA844205DA300033
:1004C0002041C007F6D50025F0E7F1BDFFFF000091
:1004D000FC70002054700020F3B583B0140001F0CC
:1004E0002DFA070001F022FA06002100049801F01D
:1004F00063FA400003990D5E8A480021405EA842DD
:1005000071DA0498401E019007D4210001F054FADA
:1005100040000399085EA84265DA0498401C0090E8
:10052000B84207DA210001F047FA40000399085E5B
:10053000854258DB601E08D4611E049801F03CFA25
:1005400040000399085EA8424DDA2000401CB042EA
:1005500009DA2100491C049801F02EFA40000399A1
:10056000085E85423FDB019800280AD4601E08D44B
:10057000611E019801F020FA40000399085EA8422C
:1005800031DA019800280DD42000401CB04209DA6D
:100590002100491C019801F00FFA40000399085E00
:1005A000854220DB0098B8420ADA601E08D4611E3A
:1005B000009801F001FA40000399085EA84212DA9F
:1005C0000098B8420DDA2000401CB04209DA641CE1
:1005D0002100009801F0F0F940000399085E85427F
:1005E00001DB012000E0002005B0F0BD0800005153
:1005F0000A710020F7B588B008A8007809A9097821
:10060000401A01F071FC060008A8407809A9497851
:10061000401A01F069FC0400B44200DA300007908F
:10062000022801DA012078E0022008A9085E0221F0
:1006300009AA515E884204DA08980090099801904E
:1006400003E0099800900898019002206946085E2E
:1006500062490968090C0907090F02004A431100A1
:10066000C911471A01256846007969460978884208
:1006700001D3069502E00020C043069001A840780F
:1006800069464978884201D3059502E00020C043BD
:100690000590049500E06D1C079885423CDA28001F
:1006A000002E01D1002003E0711E814200DA080013
:1006B0002900002C01D1002103E0621E8A4200DAE9
:1006C0001100069A424303920598484302906846F7
:1006D00040780299411868460078039A801801F022
:1006E0006BF940000A99085EB84213DB20003043E2
:1006F000D1D1A642CFD001A840780299411A6846CC
:100700000079039A801A01F057F940000A99085EAF
:10071000B842C0DA0020049004980BB0F0BD00008D
:100720008B7000200071002037710020387100208C
:10073000F1B582B0080011006A46030013700B0087
:10074000537001F039F940000299085A694648800F
:1007500000242646224D234F00E0641C3878844252
:1007600008DA029A0099A0002858FFF743FF0028F2
:10077000F3D00126002E03D1397808000A280BD1C6
:10078000A00028180221415E02226B469A5E914227
:1007900008DA0099016005E0491C39700400A000E6
:1007A00000992950A00028580090641E02E00168BA
:1007B0004160641EA0002818002C06D402216A465D
:1007C000515E0222825E9142F1DA009941603878EE
:1007D0000A2801D10120FEBD0020FEBD5870002076
:1007E000947100203E710020F3B593B000270C9760
:1007F0000B970A9702E00A98401C0A900A98484909
:10080000497A884200DB04E28000464908180178F2
:100810000391417802910221405E0690029903986B
:1008200001F0CAF811900A98401CBF490870039A59
:100830000A71029A4A710699BC4A1268120A120792
:10084000120F51434911B84A11810699B74A1268EB
:10085000120D5207520F521C1141B34A51811146D9
:10086000069A4A610299069A5143AF4A1161039967
:10087000069A5143AC4AD160114601228A613A007E
:100880004A708A700299039A1201A94B9A180001C2
:10089000505401200190064600900546044600E0B1
:1008A000641CA248006800090007000F844200DBB6
:1008B000EBE005970F970E970D9703980199401A53
:1008C000099002980099401A04900198A04202D021
:1008D0000098A04210D1049A0999139800F0DDF90C
:1008E000002809D00198A04201D10120059000986C
:1008F000A04201D101200F90029840190890019860
:10090000A04201D0A54217D1089A0999139800F086
:10091000C4F9002810D00198A04205D1012004E0BC
:100920003571002094710020380005990818059051
:10093000A54201D101200D90039880190790A6428D
:1009400002D00098A04213D1049A0799139800F09E
:10095000A4F900280CD0A64201D101200E900098E5
:10096000A04201D1012000E038000F9908180F9033
:10097000A64201D0A54216D1089A0799139800F013
:100980008CF900280FD0A64201D1012000E03800E8
:100990000E9908180E90A54201D1012000E0380000
:1009A0000D9908180D900198A0420AD1099B089A48
:1009B0000499139800F05DF9401E8041C043C00FB8
:1009C00000E038000599081810900098A0420AD15C
:1009D000049B079A0999139800F037F9401E80414B
:1009E000C043C00F00E038000F9908180590A642D8
:1009F0000AD1079B089A0499139800F03AF9401E0F
:100A00008041C043C00F00E038000E9908180490E0
:100A1000A5420AD1089B079A0999139800F015F985
:100A2000401E8041C043C00F00E038000D990818F7
:100A30001099012901DB012100E03900019A5118C8
:100A400001910599012901DB012100E03900009A9B
:100A5000511800910499012901DB012100E03900BE
:100A60007618012801DB012000E038002D180198DC
:100A7000844200DA14E70098844200DA10E7B442B6
:100A800000DA0DE7AC4200DA0AE728484068264958
:100A90008969020052085207520F914200D2AAE619
:100AA0000100C905C90F17D01F4989780200120E2D
:100AB0001207120F91420FD30699A84A0023D25E63
:100AC000914200DA97E6184989690200120D12076F
:100AD000120F914200D28EE60100C907C90F0AD059
:100AE000114A926903001B091B071B0F9A4292418E
:100AF000D243D20F00E03A00AC4B1C78032C1AD141
:100B00005B790A4C646AE40D6407640FA34212D156
:100B100000290FD004498969000F103081429241A9
:100B2000D243D20F07E000BFBC71002058700020F4
:100B3000847200203A00002A05D009200B99401A3F
:100B4000491C0B9103E00C980146491C0C910001D3
:100B500097490C1897484078E0719648C068800221
:100B60001C39496901F0C4F920809248006980026B
:100B70009049496901F0BCF960808E484069800263
:100B800011994900149A515A01F0B2F9A08089488C
:100B90008069A07103980199401A01D503980190CA
:100BA00002980099401A01D50298009000F0C6FE04
:100BB00003998919814204DB00F0C0FE0399461AAB
:100BC000761E00F0B3FE02994919814204DB00F061
:100BD000ADFE0299451A6D1E0198207330006073B6
:100BE0000098A0732800E07301988019401EA0723D
:100BF00000984019401EE0726E48807820726D485F
:100C00000078401E60720C980B9940180A2800DA90
:100C1000F1E569480B9941700C990170380003E0C7
:100C2000664902000A54401C634909788842F7DB90
:100C300005E009203900401A6149C8557F1C5E480B
:100C400040788742F5DB15B0F0BDF8B5060014001A
:100C50000020491C0D0009E00700009A290030001F
:100C600000F01BF80100380040186D1CA542F3DBB2
:100C7000F2BDF8B5060014000020491C0D0009E083
:100C800007002A000099300000F007F80100380042
:100C900040186D1CA542F3DBF2BDF8B505000F004E
:100CA0001400002F34D400F049FE874230DA002CC3
:100CB0002ED400F03BFE84422ADA2100380000F0F6
:100CC0007BFE40002D5E3B4E0820305E854211DAEF
:100CD000BA480221415EA9421ADA0021405E8542EB
:100CE00016DA3801BF49081880210155B078401C38
:100CF000B0700DE023003A007179307900F030F8DF
:100D000000902100380000F037F80099884201DA9D
:100D10000020F2BD3801B3490818015D002902D155
:100D20003178015501E0FF2101557069401970616A
:100D3000F0686F43C019F06030696C43001930618E
:100D40000A20305E854201DB012000E00020B1690D
:100D50000818B061009870700120F2BD0871002081
:100D600070B50C001D00801A01F0BEF80600601B73
:100D700001F0BAF8301870BDF8B507000E00FF2575
:100D800000240DE0A000A849081833003A0041787B
:100D90000078FFF7E5FFC0B2A84200D80500641C48
:100DA000BD4800788442EDDB2800F2BD7876002053
:100DB000D8710020BC7100203571002080710020A6
:100DC0008A710020F0B585B0B4484078002854D02E
:100DD000B2480078002850D000273E4607E0B742CE
:100DE00003D0AF4869460978C1557F1C761CAB48D3
:100DF000007886423FDAAA48805D694608706846F6
:100E000000780001A74908180190C079401C4000F3
:100E1000C0B20290FF25002400E0641C9F48407887
:100E2000844219DABA48005D00019E490918019808
:100E3000407A80007C4A1018497A890051184B7812
:100E40000A7841780078FFF78BFFC0B2A84200DA39
:100E500005000298A842E0DB0298A842BFDB8F4859
:100E60004078AB496A4612780A548C484078401C56
:100E700055394870BAE78948077088484078002893
:100E800000D198E001200290A14800780001854936
:100E90000918A0488A88C2808A7902814A7A920019
:100EA000614B9B181A785B7814000D7B641B0470EF
:100EB0001C008D7B641B44704C7B12198270C97BB3
:100EC0005918C170022101910299744A52789142D5
:100ED00067DA0021039101225CE0019989B2114196
:100EE000C90756D48A49895C09016E4B59184B7A57
:100EF0009B004D4CE3181D785E782B000C7B1B1B70
:100F000034008F7BE41B4F7BED196F463D70CD7B2A
:100F100075196E46757085786D1CDBB29D4238DBA5
:100F200005783678761CAE4233DBC678761CE4B2A0
:100F3000A6422EDB6E467678761C4778BE4228DBCA
:100F4000029E761C029601260396019F96403E4320
:100F5000B6B20196AB4200D92B00037043789C4295
:100F600000D91C00447083786C462478A34200D2D8
:100F700023008370C3786C466478A34200D22300B8
:100F8000C370C3888C881B19C38003898979591859
:100F90000181521C414949788A429EDB039900290C
:100FA00092D181780278891A491C0171C1784278FE
:100FB000891A491C417105B0F0BD00000471002080
:100FC00038B505000C00B1480078400708D5280066
:100FD000FFF759FA21002800FFF706FCFFF7F2FEA1
:100FE00031BD00008472002080B5834883490978B0
:100FF000002910D082490A781300DB07DB0F037049
:10100000096849084906490E41700C224149001DF2
:1010100000F085FF01BD4178002902D0491E4170D2
:1010200001BD0021017001BD9471002038B5984CBC
:101030000A220021200000F0D3FC0A22002195485A
:1010400000F0CEFC94480068C10715D5800F0DD084
:101050009249124A12784B789A4207D20A78904203
:1010600002D3521C0A7031BD0020087000F09EF8B7
:1010700000F052F80028FBD1002500E06D1C074865
:101080000078854207DA605D0028F7D1280000F07B
:10109000CCF80028F2D131BD3E710020357100201E
:1010A00080710020D871002070B500242500260032
:1010B0000BE0300000F0FAF8002805D0B54202DA63
:1010C000A648815D41556D1C761C754801788E429D
:1010D000EFDB0570200004E0002A00D0521E8A7069
:1010E000401C0A2813DAC100091A8900C84A51189D
:1010F000694A1368DA0702D422008A70F0E78A7816
:101100009B0D1B071B0F9342E6D21A00E7E770BD49
:101110008A71002078720020F0B482B00020009024
:10112000604902000300040017E05A4E765D002E6D
:101130000DD16700BC46AE007719BF005A4EF619B4
:101140006746F65B8E4202D222002B0031006D1CF6
:10115000534E3678B542E8DB641CAE4D2D78AC4278
:1011600005DA4B4D2D5D002DF6D10500F0E74A481C
:101170000068000A8006800E0002884213DB02200D
:10118000434904008C540A31C854AF48C05CC100C4
:10119000081A80009E490818AC49895C4170FF21FB
:1011A0008170012000900098F6BC7047F8B50024CB
:1011B0001AE06F00A000001980003B490E18A348F8
:1011C000405D0001A24909189F48005DC200101A45
:1011D00080008F4A101800F015F8F0536D1C8D48F0
:1011E00000788542E5DB641C2D480078844201DAF2
:1011F0000025F4E7F1BD000068760020367100207C
:101200006470002070B505000E00A88A3188401A6D
:1012100000F06AFE0400E88A7188401A00F064FE5B
:1012200001002000401880B270BD38B51C490A7812
:101230000A2A28DA0122CB1C14001C54834B1D18E7
:1012400028780001583318188088134B1B685B08F6
:101250001B071B0F1B01984213DB0C782000401C5E
:1012600008700C48025500F0D7F8774902000A557B
:10127000C100081A80006649081829784170FF21CA
:101280008170012032BD002032BD00003471002089
:101290006874002072740020607000206474002064
:1012A00065740020FFFF000088740020F8B52B490A
:1012B000095CCA00511A8900554A54182600361D87
:1012C0009849085C002803D0022830D01BD37BE06B
:1012D0002078022814DB944908680100490949076D
:1012E000490F0901228991420ADA800E0007000F96
:1012F000A178884204D2A08A3080E08A708063E0BE
:101300000020207060E001202070607800015049CA
:101310000D1810222900300000F001FE2888A0825C
:101320006888E08200200100218360834CE06078BF
:10133000000147490D182078012811D102202070A2
:1013400028883080688870803088A18A401A20837D
:101350007088E18A401A60832EE000BF7C74002010
:101360002A8803207049A38A9B1A0F68BF0B074085
:101370003B41D21832806A88E38A9B1A0F68BF0B00
:1013800007403B41D21872801822A25E3388A78A98
:10139000DB1B9B1A0F683F0C07403B41D21822838E
:1013A0001A22A25E7388E78ADB1B9B1A0968090C64
:1013B00008400341D0186083A888B080A879B07134
:1013C000E879F071687A7072207800281DD037882B
:1013D000758800F0B3FA860200F0A8FA800218219E
:1013E000615E79181A22A25EAA18002901D500268A
:1013F00002E08E4200DD0E00002A01D5002002E04E
:10140000904200DD1000A682E0822078F2BD00004C
:10141000507500203571002018B4FF210020C04312
:101420000022AB4C00E0521C0A2A0ADAD3009B1AB5
:101430009B00E3189B788B4201DA19001000002909
:10144000F1D112BC704700007C7400208071002034
:10145000D871002078B40F20BE49BF4A1378002B02
:101460000CD1BE4B1B78002B08D10B78034205D161
:101470004B785C1EA441E443E40F00E001247F2389
:101480000D781D40E4012C430C70B54D2600F60983
:1014900003D02E68761C2E6001E000262E602D6899
:1014A000032D01DA23400B7012780B78F0241C40D6
:1014B000024022430A70A94A12784A70B94A127847
:1014C0000B78BF241C40920140231A4022430A702B
:1014D000002203E05D71A4799C71521C0B780340DB
:1014E0009A421DDAD3009B1A8C1CE318AE4CA41848
:1014F00025781D702478E5002C1BA400744D2C1950
:10150000241D25885D702D0A9D706588DD702D0A6B
:101510001D71A588AD08FF2DDCDDFF255D71DAE7C3
:1015200071BC70477274002060700020F9B581B002
:101530000F001400002511E03100280000F03CFAF3
:101540004000395A019A125E029B1A41891A2152AF
:10155000761C00F0EBF98642EEDB6D1C00F0E3F93F
:10156000854201DA0026F4E7200000F001F8F7BD1B
:10157000F1B582B000246846214601808B4F0D46AC
:101580000846019002E00198401C019000F0D6F955
:101590000199814219DA002603E0B84200D8070019
:1015A000761C00F0C3F98642EDDA3100019800F0B4
:1015B00003FA40000299085A24186D1C69460988EC
:1015C0008142EAD269460880EAE7002603E0B84291
:1015D00000D80700761C00F0ACF986420EDA300025
:1015E00000F0F4F940000299085A24186D1C69466D
:1015F00009888142EBD269460880EBE76C4E684669
:10160000008830807780F5802000ADB2290000F09E
:101610006FFCB080C8480F21B28843680B40534329
:101620001A00D2113281B28843681B090B40534320
:101630001A00D21172810722B3884468640A1440E8
:101640005C432300DB113383B3888468240B0C4094
:101650005C432300DB11B381B388C468640A224071
:101660005A43D21153423382B288C3681B0B0B40DA
:1016700053431A00D21153427382B288C3681B0CC1
:101680000B4053431A00D211B282B28803680B4058
:1016900053431A001212F282B288C36A1B0C0B4029
:1016A00053431A00D21153427383B288C36A1B0A90
:1016B0000B4053431A00D2115342F383B288C06ADD
:1016C000000B014051430800C0114142B183F7BDF6
:1016D0005075002010B5AB49097801240A00520862
:1016E00023001A4202D000F03DF805E0C9082200AC
:1016F000114201D000F05EF8A3480178012907D11A
:10170000C178A24A1268520F914219D1447017E071
:1017100002290AD1C1789D4A1268120D5207520F50
:1017200091420DD1022141700AE0042908D1C1780B
:10173000964A1268920E5207520F914200D144709D
:101740000179002902D0491E017110BD0021C1702C
:10175000017010BD8C70002065740020377100206E
:10176000AC4500208848017800290DD101210A00EC
:101770000270874A12888281C17084490968090908
:101780000907090F01717047012909D18049828930
:101790000B881A4204D0C278521CC2700988818119
:1017A00070470000687600207C740020FFFF000076
:1017B000F4700020F1B582B000252F466846294616
:1017C00001800E4627E03100200000F0F5F84000CF
:1017D0000299085E6F4904228A5E904209DA022269
:1017E000895E814205DA6D1C01990122A2400A43FB
:1017F0000192B84205DA07006846210041703100C5
:101800000170641C00F09AF88442DCDBB00062498D
:10181000019A0A50761C00F089F8864203DA00200B
:1018200001900446EEE7584C5A480021405E87423A
:1018300031DA2078002811D10220207027816846F3
:101840004078A07268460078E0720120E0704F484E
:10185000006800090007000F2071F7BD022861D160
:10186000A07A69464978401A00F03EFB02280ADA5D
:10187000E07A69460978401A00F036FB022802DA5D
:10188000E078401CE070278168464078A072684686
:101890000078E072F7BDADB2002D22D03B4E30682B
:1018A00000090007000F207100F040F882003A495B
:1018B0003A4800F034FB2078002805D1032020703E
:1018C000E58001206071F7BD03282BD16079316874
:1018D000C90D4907490F884201D2401C6071E5805B
:1018E000F7BD2078002811D1042020702781684698
:1018F0004078A07268460078E0720120E0702348CA
:10190000006800090007000F2071F7BD042809D105
:10191000E078401CE070278168464078A0726846F5
:101920000078E072F7BD1E48007870471D480078C7
:1019300070471D48007870475070002010B5FFF7C1
:10194000F2FF0400FFF7F5FF012801DB012000E0B2
:101950000020201A10BD1549085C70471449085C26
:10196000704780B5FFF7DFFF10490818401E007868
:1019700002BD1049085C704780B5FFF7FAFF0C49BB
:10198000085C02BD34710020787600207C70002055
:101990003C7100200E7100204071002088760020EC
:1019A00000700020017000200270002004700020F0
:1019B000247000203470002038B50C00FFF7CBFFF6
:1019C00005012000FFF7CAFF281832BD38B5040012
:1019D000FFF7C7FF05012000FFF7CEFF281832BD33
:1019E00010B5040010000A000100200000F0B2FA57
:1019F000200010BD0121C006C00E81409A48016040
:101A0000704780B500F01AF800F0D7F800F069F8D8
:101A100000F081F800F091F800F0B5F800F0DEF881
:101A200000F0FCF900F00AFAFE20400000F0E9F9AD
:101A300000F0ECF90320FFF7DDFF01BD9E480168CF
:101A400004220A4302607047A220C00501680122F7
:101A50000A4302607047A220C005016802220A43BF
:101A6000026070479B48016801220A430260704788
:101A700098480168012291430160704787490A68CC
:101A8000A44B13400007C022920502401A430A608B
:101A9000704782490A6852005208C30713430B601B
:101AA0000A689D4B1340400880078022D2051040F1
:101AB00018430860704788490860704786490A687B
:101AC000AB4B13400004FF22120402401A430A6089
:101AD000704781490A68FF239A43C0B210430860E7
:101AE00070478E4801681F22914305220A43026015
:101AF000C1698B4A0A40A82189021143C161C16AA8
:101B00007F229143C162C16A9E4A0A408021C90175
:101B10001143C162704710B5002000F01FF89024F7
:101B2000E40022000021FFF75BFF012000F016F81F
:101B300022000021FFF754FF10BD10B5002000F077
:101B400013F8AB4C22000021FFF74AFF012000F000
:101B50000BF822000021FFF743FF10BD002801D041
:101B600089487047A8487047002801D0864800E09F
:101B7000A5488021090140187047BC480168080049
:101B8000C007C00F7047A4480168AB4A0A4302600F
:101B90004168B94A0A43426070479F490A68120C7B
:101BA000120402430A607047B4490A68920F920710
:101BB00080008008104308607047AB4801688022AD
:101BC00012020A4302600168A94A0A400260AC4856
:101BD0000168802212040A430260704780B5012028
:101BE000FFF76CFF1420FFF774FF012000F030F8BE
:101BF000A04800F055F80120FFF74BFF00F0FAF87D
:101C000000F014F800F016F8002000F018F800209A
:101C100000F0A1F800F0AEF80021084600F0B6F898
:101C200000F0DAF8974800F0E9F801BD96489749C6
:101C3000016070479648D2210904016070479549B8
:101C40000A6810239A430001184010430860704747
:101C500012490A68904B13404004F8229203024054
:101C60001A430A607047000000E100E010B40B491D
:101C70008A6910239A4303005B091B011024234047
:101C800013438B610A68844B13404004F82292038B
:101C900002401A430A6010BC704700000400005163
:101CA0007E490A68520C52040A600A68C003C00BDD
:101CB00010430860704700002020004877490A68F8
:101CC000774B13400002F022120102401A430A60CF
:101CD00070470000480000511000005138B5714AAB
:101CE0001368714C1C40030680256D042B40234370
:101CF000136000280CD01068000A8005800DC00019
:101D00006A4A8018F0220B011943C9B2FFF768FE36
:101D100031BD0000FFFFFFCFFFFFFFBF14000051E8
:101D2000FF00FCFF10B55F4A1268120A9205920D7F
:101D3000D2005E4BD3180001401008220C01214351
:101D4000C9B204006410A40F201880108000181875
:101D5000FFF746FE10BD56494A6803239A438007A1
:101D6000800F104348600020C043086070470000A7
:101D7000FFFF00FF4F4850490160504941608160BA
:101D8000C1607047FF80FFFF0090002030B4494AD7
:101D900013684B4C1C408B03F025AD021D402543BE
:101DA00015601368474C1C404302F825AD011D40E7
:101DB000254315601368444C1C404901F0235B0027
:101DC0000B402343136011681F239943C006C00EC4
:101DD0000843106030BC7047324801683F2291438D
:101DE0000A220A43026001682F4A0A4002607047D3
:101DF0001C040000354836490160704735490860C9
:101E00007047354908607047008000203348002142
:101E1000C9430160704700000800005180B52B489D
:101E20000068C006C00E0002204940188C222C49D0
:101E300000F075F801BD0000FFFF000080B5002133
:101E40000846FFF74BFF01BD264800680100090A5C
:101E50000800C007C00F70471E4800680100890EC7
:101E60000800C007C00F7047680000519000005183
:101E7000FFCFFFFFAAF80100FFFFFF3F0C0000515A
:101E800024200048334455003400005140362301DB
:101E9000380000511C000051FFFFC1FF0400005139
:101EA000FFF0FFFF30000051FFFFFFFE0080002029
:101EB000180000512000005100003C0A26330404A1
:101EC000FF3FFCFFFFC1FFFF1FFEFFFF140000519B
:101ED00005008B0D3C00005174000051780000514A
:101EE000C04400207C000051002800D540427047CB
:101EF000094210D088420BD30122002300185B4115
:101F00008B4200D35B1A5241F8D31900100070477E
:101F100001000020704708B500F046F808BD10B574
:101F2000040000F043F8200010BD38B40121002265
:101F30000368001D002B0BD00468001D0C4202D06A
:101F40004D466D1E64192260241D1B1FF0D0FAE758
:101F500032BC70471206130A1A43130C1A4300BF0F
:101F6000094205D0830705D00270401C491EF9D1F3
:101F700070470000130030B414001500103902D36C
:101F800010393CC0FCD2490700D30CC000D504C0B6
:101F9000890002D30280801C002900D5027030BC69
:101FA000704700000022E5E770470000124207D0AA
:101FB0008B0706D00B78491C0370401C521EF7D8C3
:101FC0007047830706D00B78491C0370401C521ED3
:101FD000F9D1704770B4103A03D378C9103A78C079
:101FE000FBD2530701D318C918C001D508C908C0CE
:101FF000D20704D30B880380891C801C002A01D5DA
:102000000B78037070BC704730B58BB01D48182139
:1020100001700D2141700321817005A81AA11822B9
:10202000FFF7D8FF01A800BF1DA11022FFF7D2FFC4
:10203000684600BF1EA10A6802600024250004E073
:10204000A94805A9495D41556D1CFFF76CFC854207
:10205000F6DB250004E0A54801A9495D41556D1C4A
:10206000FFF764FC8542F6DB04E0D7486946095D6A
:102070000155641CFFF75DFC8442F6DB00F064FB55
:102080000BB030BD007000200F0E0B0A07060504D0
:1020900003020100101112131415161718191A1B38
:1020A00000010203050708090A0B0C0D0E000000D1
:1020B00002060A00F0B4A9490868000C0004086090
:1020C000C24A0240A020400310430860486882B220
:1020D000C820800310434860FF22904364230343D9
:1020E0004B609F4A1340480D184348600F20C0437F
:1020F0008C680440032323438B60B54D1D400C0CBA
:102100002C438C60F023DB431C40202525438D604D
:10211000CD68054005242C43CC601C401025254388
:10212000CD604C0D2C43CC60AA4E2640A0252D013D
:102130003543CD60A84C2540CE0B2E43CE600D69B3
:1021400028400A2505430D611D40402028430861B1
:1021500010400D0D05430D612540A020C00128430E
:102160000861C54D0540C020000328430861B64DF5
:1021700028408026760306430E6101264F693743C7
:102180004F610E2087430420384348611840C02720
:1021900007434F61480D384348618E4F0740080D93
:1021A000384348612040A027FF0107434F61B248F0
:1021B0003840F70407434F61B0483840B70507433C
:1021C0004F61AF483840770607434F613801000937
:1021D000B70707434F618F6937438F611E208743DD
:1021E000182038438861E027B843C02707438F6130
:1021F000B44838404F0C07438F61B3483840CF0B89
:1022000007438F61B1483840370407438F61B048B6
:102210003840B70407438F61AE483840A0277F0499
:1022200007438F61AC483840F70607438F61C020F1
:10223000000638438861C8693043C861FE27B84347
:1022400014270743CF610F6A37430F62402087434B
:102250000F623E2087430F625D483840E827BF0188
:1022600007430F6259483840F70507430F62D00B08
:102270004862B0488862B048C862B0480863B04855
:102280000863486B06434E630E20304348630340A7
:10229000A02018434863784B0340A0200003184354
:1022A000486305408020C003284348630240080D6E
:1022B0001043486304408020000220434863BE4A24
:1022C0000240A020800410434863C74A0240A02077
:1022D000400510434863C000C008C022D205024335
:1022E0004A63F0BC70470000047000202470002096
:1022F00038B5BE4D03202873002001006973297290
:10230000012129746974A9740100E974E88110221B
:10231000B748FFF765FBB74C0C2200212000FFF700
:102320005FFB2078FFF717FBA0706078FFF716FBC4
:10233000E0702868C003C00BA06000F0F6F920220E
:102340000021AD48FFF74CFB00F09CFAFDF7BEFE04
:10235000FDF7C4FEFDF7CFFE31BD00004870002040
:10236000FFF0FFFF38B5FFF776FBA448017E01249C
:102370000268224003D104220A43027631BDFB22C7
:102380000A4002769A4D10004009210008420DD003
:10239000102200212800FFF723FB0020FFF76EFB2F
:1023A0002046FFF78BFB0020FFF7D5FC2878800044
:1023B000CC490D182868400C04402000FFF73FFC72
:1023C0002868FFF76DFC31BD34700020FFFF00FF6F
:1023D000FF00FFFFFFF1FFFFFF0FFFFF38B5FFF723
:1023E0003AFB824C207A01252168490C294003D10F
:1023F00004210143217231BDFB2101402172284695
:10240000FFF73CFB2846FFF759FB20680100890CC9
:102410000D400CD0C00CC006C00EFFF79CFA0500A2
:102420002068000E0007000FFFF798FA05E0002073
:10243000FFF791FA0500C04800780100C9B22800F2
:10244000C0B2FFF7A3FC31BDFFFF8FFF10B5BB4C3F
:10245000207880060ED5FFF7FEFA2078FB21014098
:1024600021700220FFF70AFB0120FFF727FBB44889
:10247000FFF7C4FC10BD0000FFFFF0FFFFFF0FFFE0
:10248000FFFFFFF010B5AD4C2078800618D5FFF7A0
:10249000E2FA2078FB2101402170FE204000FFF786
:1024A000B0FC0220FFF7EAFA0020FFF707FBA5487F
:1024B0000068000CC0B2FFF70CFBC648FFF79EFC9B
:1024C00010BD0000FFC0FFFFFF3FFFFFFFFFFCFF4D
:1024D000FFFFC3FFFFFF3FFCFFFFFFC338B5474CC3
:1024E0002068012528420ED14008C006C00EFFF723
:1024F000AFFB2068800905402800FFF7A0FBCC480F
:102500000021017031BD7034206D800B80B2002835
:1025100005D02078022802DA401C207031BD00F07E
:10252000C7F9FDF7EFFD6078FFF7A0FBC048002179
:10253000017031BDFFF80100FFF10100FFF8030059
:10254000FFF8031038B5294C206801008903C90F32
:1025500004D1FFF7A5FB0020607431BDB5480168C8
:1025600061670F250068000C2840A16FC94A0A4026
:102570000102280208401043A067FFF791FB206882
:10258000000F15D0A06F000A054029000120FFF7B9
:10259000A5FB2068000F2D1A280040B2002800D5A6
:1025A0000025FFF7DEF92900C9B2C0B2FFF7BAFB78
:1025B0000020607431BD0000FFFF7FFC10B50020DB
:1025C000FFF7CCFA04000020FFF7CEFABB4A210047
:1025D000FFF7A5FC0020FFF7C7FAFEF7C9FFBB48CD
:1025E0000021017010BD0000FFFFFFE378700020A4
:1025F000D8700020E870002014710020687000205E
:1026000080B5FFF72FFA00F01AF8002000F0EFFB7A
:1026100000F021F8012000F0EAFB00F026F802208B
:1026200000F0E5FB00F029F8032000F0E0FB00F0EB
:102630005BF8042000F0DBFBFFF71AFA01BD10B5D0
:10264000FDF744FD00F03CF9040000F031F92100F1
:10265000FDF7FAFD10BD10B500F032F9040000F0EE
:1026600027F92100FEF7ACFC10BD80B5FEF7DEFCBB
:10267000FEF71AFDFEF7B8FC01BD10B50120944924
:102680000A78024202D09349487010BD4A78002A65
:1026900005D18A78002A02D1C978002908D08E494C
:1026A000096B49084907490F88408A49887010BD5D
:1026B000884CA078002802D0401EA07010BD00F009
:1026C000F7F8FFF707F884482178002903D001685C
:1026D000090C418710BD418F002901D0491E418757
:1026E00010BD00006C70002010B5FEF7B3FE7B48F3
:1026F0000278002A18D00121794B1C680C4003D0C5
:10270000012A01D10C0000E00024494A14701B6921
:102710005B0C0B4002D00378012B00D000215170DC
:1027200000789070FDF7E7FC10BD80B548220021CD
:102730006C48FFF755F901BDDD7000208070002066
:102740003344550048700020F8B500252C002E00B9
:102750000BE0270001210C003000FFF7FCF82100FE
:1027600081403C0021430C00761CFFF7DCF88642D8
:10277000EFDB2F0008E001262800FFF7EFF8864086
:102780003E43B6B237006D1CFFF7D0F88542F2DB4E
:102790002000FFF709FA3800FFF7FFF9F1BD10B587
:1027A000514C2078C00613D5FFF755F92078FB214E
:1027B000014021700120FFF724FB0220FFF75EF9A2
:1027C0004548006880B2FFF776F90248FFF716FB2C
:1027D00010BD00003344550470B544480178F8201A
:1027E0000840434C2070002803D100F061F8FDF749
:1027F000FBFD207800281AD13E4EF08E002802D032
:10280000401EF08670BD3068000AC0B2F08600F04D
:1028100057F8050000F054F8040000F049F831685A
:1028200009090B071B0F2A002100FEF77FFE70BD70
:10283000887000208400005180B52F48017800295D
:102840000ED12E494A68C2600A6842600A698260F5
:102850004A690261CA6942610A6A8261496AC16160
:102860000178491C0170FFF7D1FA01BD22480078B8
:10287000704721480178022901DB012141700021C4
:10288000017070471E480021017041708170C17055
:1028900070470000FFF0FFFF10B5FFF76EF9401E14
:1028A0008041C00F164C2070FFF767F9A07010BD73
:1028B00080B513480078FFF751F902BD1C040000F1
:1028C00080B510480078FFF74FF902BD8A700020EC
:1028D00034710020787600204C700020797600203A
:1028E000687000208C70002080700020187100201B
:1028F0008B70002050700020147100206C0000517B
:10290000D4700020D570002080B5E82200219C48BA
:10291000FFF766F8012000F004F8002000F030FA1C
:1029200001BD97490870E020C00088800020C88061
:10293000704780B592480078012802D0022803D061
:1029400004E000F01EF801E000F02FF800F0BCF900
:1029500001BD80B58A480078032806D010D3052829
:1029600009D005D3062809D001BD00F050F801BDFB
:1029700000F067F801BD00F099F801BD00F0C1F862
:1029800001BD80B5FFF794FF7E490A681300DB059F
:10299000DB0F03D18968090A890705D19022D2008B
:1029A0000100B348FFF7BBFA01BD38B5FFF780FF60
:1029B0000400B04D69782878401EFEF7FDFF400006
:1029C000205A00F0B5F86978491E2878FEF7F4FF20
:1029D0004000205A00F0ACF869782878FEF7ECFF48
:1029E0004000205A00F0A4F86978491C2878FEF7C6
:1029F000E3FF4000205A00F09BF869782878401CDB
:102A0000FEF7DAFF4000205A00F092F831BD38B5E9
:102A10005C4C607E002813D000F079F82068C0B2CA
:102A200000F075F8002508E01021A148405D000184
:102A3000A04A101800F08DF86D1C607E8542F3DB13
:102A400031BDF8B59C4F387800282ED000F05FF8E3
:102A50004C480068C0B200F05AF8002422E09748C1
:102A6000005DC100091A8900954A55186978090165
:102A7000904A561800F04BF8A87800F048F83088D3
:102A800000F056F8708800F053F8A88800F050F86D
:102A9000E88800F04DF8288B00F04AF8688B00F0C9
:102AA00047F8641C38788442D9DBF1BD70B5854C99
:102AB00020780100C90923D000F029F8314D286899
:102AC000C0B200F024F8607800F021F80F262078DA
:102AD000304000F01CF8E87E00F019F876480078E5
:102AE00000F015F8002507E00721E800401BA21CB4
:102AF000101800F02EF86D1C207830408542F3DB72
:102B000070BD80B520219C4800F023F801BD010074
:102B10009A4A53881088834204D21800401C50807F
:102B20005348C1545188128891428041C00F704768
:102B300092494A880B885B1E9A4204DA4C4B9852A1
:102B40004888801C48804A8809888A428041C00F92
:102B5000704738B50D00894C63882188491B8B422A
:102B600008DA2A0001004248C018FFF7D8F9608847
:102B7000401960806188228891428041C00F32BD37
:102B8000C87600201C710020F8B5954F09203870D8
:102B90000024250000E06D1C032D62DA26000AE007
:102BA000FEF7C4FE401E2901491B89008D4A5118B9
:102BB00029310870761C032EEDDA002D03D0022D8A
:102BC00016D007D31EE0B00080198000854922008E
:102BD0000A5417E0FEF7B2FE0100C90F08184010B2
:102BE000B100891989007F4A51183C31087009E009
:102BF000FEF7A4FE401EB10089198900794A5118D8
:102C000078310870002E03D0022EC9D008D3D1E746
:102C10002801401B80007349081821004170C9E752
:102C2000FEF784FE2901491B89006E4A5118491C90
:102C30000200D20F101840100875BBE7A000001961
:102C4000800068490D182878FEF785FEA87068781E
:102C5000FEF784FEE87069782878FEF7ADFEA8805C
:102C6000641C38788442E9DB8020B880F1BD000024
:102C700000790020D07600205B480178002900D13F
:102C8000704718B4002211000BE08B005B189B000A
:102C9000544CE3181400DC80DA601A611C815C81FA
:102CA000491CC3799942F0DB401C028111BC70477A
:102CB00080710020D8710020657400207C74002091
:102CC000507500208C70002049480068000F800774
:102CD000800F022800D07047F8B5434C20780028B8
:102CE00048D0641C2089641E641C6189641E88426B
:102CF00040D2FFF7DDFD0021641C2289641E002AFA
:102D00002FD1E27991422FDA364A8B005B189B0073
:102D1000D21893885B00C35AD3801381D388538120
:102D2000491CEEE72F4A8B005B189B00D218938852
:102D30005B00C35A1D00D688AD1B6DB2D6687619EC
:102D4000D66016692F006F43F519156115899D42EC
:102D500000D21D0015815589AB4200D92B0053814B
:102D6000491CE2799142DDDB641C2089641E401C11
:102D7000641C2081F1BD000090770020CC760020FB
:102D800010B5194C207000202072FFF7FDFEFFF7F0
:102D900073FF2078012806D01CD303281BD019D23A
:102DA0000020FEF763FF0220FEF768FE0020FEF71A
:102DB00085FE1048FFF722F80F480278FB211140EA
:102DC000017001220A43027002211143017008229E
:102DD0000A43027010BD0020FEF770FFE3E7000019
:102DE000D2760020D8760020CB760020704770473E
:102DF0000400005133445500807000200121C006BA
:102E0000C00E81409948016070470121C006C00E84
:102E10008140B748016070470121C006C00E814063
:102E2000B4480160704738B402009007800FC500B5
:102E3000FF242000A840C34388010440AC40100098
:102E40000BD50007000F0838800880008849081853
:102E500001680B401C43046007E080088000A9491A
:102E6000081801680B401C43046031BC704780B5F2
:102E7000042000F061FA00F073FB182000F084FBDE
:102E80007C4800F08BFB01217B4800F0B8FB02215D
:102E90007A4800F0B4FB0021A94800F0B0FB0920FB
:102EA000FFF7B3FF0920FFF7B7FF01210920FFF764
:102EB000BAFF0920FFF7A2FF00F05FFB01BD80B55C
:102EC0000021042000F0B0FB0121042000F008FCE8
:102ED0000121042000F020FC01BD0200FF239B1C07
:102EE0009A4203DA9748006881547047E0231B0137
:102EF0009A4208DB5B1D984205D29348914B5B6870
:102F00009A181154704780235B019A4208DB8F4B5B
:102F1000984205D28E488B4B9B689A181154704783
:102F2000C0239B019A4208DB1B1D984205D28948A9
:102F3000844BDB689A1811547047874BC018A02344
:102F4000DB00984204D284487E4B1B699A181154C6
:102F500070470100FF22921C914203DA7948006811
:102F6000405C7047E0221201914208DB521D904202
:102F700005D27548734A52685118085C7047802220
:102F80005201914208DB714A904205D270486D4A65
:102F900092685118085C7047C0229201914208DB88
:102FA000121D904205D26B48664AD2685118085CDF
:102FB0007047694A8018A022D200904205D2664824
:102FC000604A12695118085C70470020704770B55C
:102FD000624C02202074A068002806D100F003FB98
:102FE000A080A068401CA06070BD012809D100F03D
:102FF000FAFAA18809020818A080A068401CA06005
:1030000070BD00F0F0FAA2881100FF239B1C9942CA
:103010001EDB1300E0252D01A94202DB6D1DAB4232
:1030200016D380256D01A94202DB484DAB420FD378
:10303000494D5D19A026F600B54209D3C025AD0162
:10304000A94202DB68498B4202D3684959180AD168
:103050000100C9B21000FFF740FFA068401CA0604B
:10306000A088401CA08070BD0000000000E100E0CE
:103070001CED00E040BF0100CF2F00208130002078
:1030800038B5364C01202074A0880100FF22921C24
:1030900091421EDB0200E0231B01994202DB5B1D13
:1030A0009A4216D380235B01994202DB274B9A4256
:1030B0000FD3294BD318A025ED00AB4209D3C02371
:1030C0009B01994202DB48498A4202D34749511881
:1030D0000AD1FFF73EFF00F07FFAE068401CE06095
:1030E000A088401CA08031BD002000F075FA31BDE1
:1030F00080E100E080E200E0184800218160C160CA
:103100000174704700E400E080B50021042000F065
:1031100003FB9620800100F05AFB01BD00B5344945
:1031200008780200D20901D1002000BD4006400EFF
:103130000870044800684822FEF738FF012000BDEF
:10314000F93000204C45002000F2FFFFB0170000CE
:1031500000F0FFFF00D0FFFF00E0FFFF74450020FC
:1031600080B524480078012831D10920FFF74DFEB1
:103170000D20FFF74AFE0320FFF747FE1E20FFF752
:1031800044FE0820FFF741FE0220FFF73EFE072025
:10319000FFF73BFE0021042000F046FA0021042046
:1031A00000F09EFA0121042000F0FAF800F0B7F9CF
:1031B00000F0BCF90020FFF721FE022000F0A6F885
:1031C00000218020FFF789FE00F083FB30BF8320C1
:1031D000FFF7BFFE012805D100218320FFF77DFE08
:1031E00000F073FB01BD00000430000000C0FFFFD1
:1031F0008C700020A445002080B5FFF7B1FFFFF7D9
:103200008DFF002801D0FFF77FFF01BD002912D0FC
:10321000402910D200280ED040280CD288420AD370
:103220005C4A13681B071B0F4903800108430343D3
:103230001360012070470020704700280BD0102831
:1032400009D254490A680F239A430007000F10431C
:103250000860012070470020704700280DD0082822
:103260000BD24D490A684D4B1340C004E022920333
:1032700002401A430A60012070470020704710285E
:103280000BD245490A68A84B13400003F0221202F2
:1032900002401A430A60012070470020704700284E
:1032A0000DD040280BD23C490A68A34B13400001C3
:1032B000FC22920002401A430A600120704700205D
:1032C000704700280BD0082809D233490A68072321
:1032D0009A434007400F10430860012070470020C8
:1032E0007047002910D08022120191420CD2002890
:1032F0000AD09200904207D2884205D3C0024018FB
:103300008E49086001207047002070478C490A6888
:1033100003239A4383079B0F13430B6089490028BB
:10332000086803D104229043086002E004220243AB
:103330000A60012070470000052829D801A1095C16
:103340008F4400BF06121E2A36427F4801680122C0
:103350000A43026070477C48016802220A43026007
:1033600070477948016804220A4302607047764832
:10337000016808220A4302607047734801681022FE
:103380000A43026070477048016820220A430260C5
:10339000704700001420004818200048FFFFC7FFB6
:1033A000F0B482B00500002906D0022956D015D30A
:1033B000032900D194E0B0E07F21C943634A072D7F
:1033C000106802D101401160A7E001400123AB4029
:1033D00098434006400E084310609EE07F21C94399
:1033E0005B4F7F23594A072D10D1106801401160AF
:1033F00010680740176010685649014011600020AE
:10340000C043506010680343136086E014681C409A
:10341000106808401060106800900126AE4035002A
:10342000EE430740BC460746300238401F020740C3
:103430006046074317601068464F07403604064051
:1034400018043040384310600020C04350601068BA
:10345000014025432B400B4313605EE0FE20C00378
:103460007F21C9433A4F7F23384A072D14680ED174
:103470002140116011680F40176011680843106007
:103480000020C043506010680343136045E01C40B7
:1034900016680E401660166800960126AE4035008C
:1034A000009E3740BC463746EE4336023E40070A90
:1034B00037406646374317601768264E3E40B4468D
:1034C0002E043E4330406646304310600020C04327
:1034D00050601068014025432B400B4313601CE0F3
:1034E0007F231802194A072D116805D1084310607F
:1034F00010680343136010E00126AE403500144C01
:103500000C402E020E433040204310601068C10969
:10351000C90105432B400B431360F3BC70470E48B1
:103520000068704700000000FF0FFFFF4006400EDC
:103530000A490860704700000FFCFFFF1C2000488C
:103540000020004810ED00E0202000483C2000480A
:10355000FF80FFFFFFFF80FF44200048402000481D
:103560002E4801680A698023DB0113430B61006860
:1035700001692B4A0A4002617047284800680169C6
:1035800040220A4302617047244909680A6A7F237E
:103590009A434006400E1043086270471F4909686D
:1035A0000A691043086170471C48006880697047C9
:1035B0001A4909688A69104088617047174800688D
:1035C000016908220A4302617047144800680169D2
:1035D000272291430161704780B5104909688860CE
:1035E000FFF7ECFF01BD10B50C4800688468016965
:1035F000042291430161FFF7E1FF200010BD04297F
:1036000002D28900074A5050704780000549085887
:10361000010000D1704780B5804701BD644500209E
:10362000FFBFFFFF98450020062853D801A2125C77
:10363000974400BF081E344A60768C002648026812
:10364000264B13404902F02252010A401A430260FD
:10365000704721484268214B13404902F022520131
:103660000A401A43426070471B4882681B4B134054
:103670004902F02252010A401A43826070471648FC
:10368000C268164B13404902F02252010A401A4305
:10369000C260704710480269104B13404902F02283
:1036A00052010A401A43026170470B4842690B4BB2
:1036B00013404902F02252010A401A434261704706
:1036C00005488269054B13404902F02252010A4025
:1036D0001A4382617047000000100048FFE1FFFFBD
:1036E00000290BD11A4909680A6A7F239A430123EA
:1036F00083405806400E10430862704701290AD1E2
:1037000013490968CA697F239A43012383405806F5
:10371000400E1043C861704701290BD10C4909685C
:103720008A687F239A43012383405806400E104342
:103730008860704700290AD105490968CA687F2353
:103740009A43012383405806400E1043C8607047D7
:103750006045002038B505002E4C0120206017E0A0
:10376000401E00F0FDF800F008F9012000F0E4F838
:1037700000F0D6F8012000F0C7F827482D1800F017
:10378000E7F80128FBD0002000F0BEF800F0CEF8EA
:10379000802040048542E3D2002D15D0280000F09F
:1037A000DFF800F0EAF8012000F0C6F800F0B8F801
:1037B000012000F0A9F800F0CBF80128FBD0002090
:1037C00000F0A2F800F0B2F80020206031BD80B512
:1037D000124901220A60110688420DD3481E00F0EA
:1037E000BFF800F0CAF8012000F0A6F800F098F841
:1037F000012000F089F801BD00F0B2F800F0BDF83A
:10380000012000F099F800F08BF8012000F07CF81E
:1038100001BD0000B0450020010000FFB4450020BC
:10382000BFF34F8F2E482F490160BFF34F8FFEE744
:103830002D490860BFF34F8F704710B58020800579
:10384000FFF7F6FF294C20682949014080208001BC
:103850000843206020680F2188430921014321602B
:10386000206810210143216001210846FFF7CEFCAA
:103870000F20FFF7E2FC0120FFF7EFFC0F20FFF71E
:10388000FEFC01211B48FFF72CFD3F20FFF707FD41
:103890000720FFF716FD206817490140C020C0022D
:1038A00008432060206815490140C0208003084378
:1038B0002060FFF7DCFAFFF702FBFEF7A2F800F04A
:1038C00069F80F48FFF746FF10BD80B5FFF7A8FF66
:1038D00001BD054800684068401E0A4908607047FD
:1038E0000CED00E00400FA0508ED00E0242000489B
:1038F000FF0FFEFFFF1F0000FFFFF1FFFFFF8FFF25
:1039000000F04902FC7F00201F490128086803D10C
:10391000012202430A607047012290430860704709
:103920001948016802220A4302607047164801687C
:10393000022291430160704713490128086803D1AE
:10394000042202430A6070470422904308607047D3
:103950000D480068C00301D5002070470120704762
:1039600080214904884201D3012070470002000AE7
:10397000401E064908600020704705480021C943E1
:10398000016070470000000010E000E014E000E07B
:1039900018E000E080B5FEF737FBFEF78BFBFEF783
:1039A000A7FCFEF7B1FF01BD10B5FEF762FF784C32
:1039B0002078C0075ED4207900280CD0032832D1AB
:1039C0007448006880B274494843FFF7C3FE002082
:1039D00000F0C3F827E06079012811D017D303283D
:1039E00007D014D2207A00281DD1002000F0C0F8A2
:1039F00019E0607A002816D1002000F0B9F812E032
:103A0000A07A00280FD1002000F0B2F80BE0614846
:103A10004068000C07D0E088002804D1012000F0A5
:103A20009CF80020E0722079002802D0012818D0EC
:103A300010BD607900281DD1207A002803D0022013
:103A400000F096F810BD607A002803D0032000F043
:103A50008FF810BDA07A00280CD0012000F088F863
:103A600010BDE07A002805D0002000F076F8002094
:103A700000F07EF810BD46480178890700D57047F0
:103A800080B50179002902D0012915D001BD407906
:103A9000002805D0022809D005D3032809D001BD8C
:103AA000FEF7F0FC01BDFEF7D1FC01BDFEF75AFCAC
:103AB00001BDFEF793FC01BDFEF771FE01BD80B5AF
:103AC00033480078400702D5FDF7C5FF01BDFEF77A
:103AD000BBF9002803D0FDF7B7FFFEF7D3FE0620A1
:103AE000FFF785F900E030BFFEF7C0FE0028FAD0EE
:103AF000FEF7D2FEFEF71DFF0720FFF778F9FFF76C
:103B000075F901BD22480178090700D5704780B5D5
:103B10000179002902D0012915D016E0407900284A
:103B200005D0022809D005D3032809D00DE0FEF7FF
:103B300067FD0AE0FEF742FD07E0FEF7CFFC04E078
:103B4000FEF700FD01E0FEF747FEFEF702FF00F082
:103B500016F80520FFF74BF901BD0D4908710F4814
:103B60000068000CC8800878102202430A70704771
:103B7000074948710878202202430A7070470448B8
:103B80000278EF2111400170DF220A400270704775
:103B9000807000204870002080BB00004C70002026
:103BA0007047FEE77047704710B52348006800284B
:103BB00032D02248006800283DD021480168002901
:103BC0001DD0491E01601DD11E4C2068002812D056
:103BD0000020FFF799FEFFF7A9FE2068FFF7C0FE5F
:103BE000FFF7CBFE0120FFF7A7FEFFF799FE0120AC
:103BF000FFF78AFE06E014480121016002E0124846
:103C00000121016010480068002814D00020FFF74F
:103C10007BFEFFF78BFE10BD0C48016800290AD01F
:103C20000021016001210420FFF776FD0020FFF74D
:103C30006BFEFFF77BFE10BDB045002088450020DD
:103C40008C4500209045002094450020B44500207C
:103C50007047704780B500F03BF800F03DF801BDBB
:103C600080B5FEF7E9FD01BD80B500F042F800F037
:103C700039F801BD704710B5FFF796FC0400FFF757
:103C800097FCDE20C00020401CD0A00509D5FFF71E
:103C90009CFCE00703D50220FFF7B7FC01E0FFF72B
:103CA0008DFCE00602D50020FFF7AFFC422020404B
:103CB000402802D10220FFF7A8FC200602D50120EF
:103CC000FFF7A3FC10BD70477047704770477047FF
:103CD000034800680069704701490968C860704777
:103CE0006845002006480068016804220A43026013
:103CF000704703480068816801220A438260704768
:103D00007045002038B401210268001D002A0FD040
:103D10000368C318446808300C4202D04D466D1E3B
:103D200064191D6825601B1D241D121FECD0F8E7C7
:103D300032BC704710B5074979441831064C7C44B1
:103D4000163404E0081D0A68891888470100A1425A
:103D5000F8D110BD0800000028000000CFE1FFFFEF
:103D600044000000744500200000000099FFFFFFA0
:103D7000B400000098000000C044002000000000D3
:103D800080B5FFF75AFDFFF70FFEFFF774FEFFF750
:103D900096FEFFF7B7FEFFF72FFAF4E700F009F8F9
:103DA000002801D0FFF7C6FF0020FFF7E9FF00F071
:103DB00002F80120704780B500F002F801BD000054
:103DC0000746384600F002F8FBE7000080B5C04621
:103DD000C046024A11001820ABBEFBE726000200D5
:103DE0000148804701480047F13D0020013E002086
:103DF00001480249016070476C45002040787D0110
:103E0000C046C046C046C046FFF7C8FF05010202D3
:103E10000202030303040404050506060707080855
:103E2000090A0A0B0C0D0D0E0F10111213141517A1
:103E300018191B1C1D1F2022232527282A2C2E3051
:103E4000323436383A3C3E414345484A4D4F52544D
:103E500057595C5F6264676A6D707275787B7E81AA
:103E600084878A8D909295989B9EA1A4A7A9ACAFB8
:103E7000B2B4B7BABCBFC1C4C6C8CBCDCFD1D3D5FD
:103E8000D7D9DBDCDEE0E1E2E4E5E6E7E8E9EAEB0E
:103E9000ECECEDEDEDEEEEEE00780020A445002018
:103EA0000070002000000051007900200040004810
:103EB000007000480022004840787D010060004802
:0400000520003E0198
:00000001FF
